:020000040800F2
:100000000004022001020008750F0008790F0008A3
:10001000CD0F0008790F0008A10F000803020008A7
:100020000302000803020008030200087927000801
:10003000030200080302000803020008030200088C
:10004000030200080302000803020008030200087C
:10005000030200080302000891390008BD390008B6
:10006000E9390008153A0008413A0008030200087F
:10007000030200080302000803020008030200084C
:10008000030200080302000803020008030200083C
:100090000302000803020008030200086D3A00088A
:1000A000030200080302000803020008030200081C
:1000B000B537000803020008030200080302000825
:1000C00003020008030200080302000803020008FC
:1000D00003020008030200080302000803020008EC
:1000E000D53A0008030200080302000803020008D2
:1000F00003020008030200080302000803020008CC
:1001000003020008030200080302000803020008BB
:1001100003020008030200080302000803020008AB
:10012000030200080302000803020008030200089B
:10013000030200080302000803020008030200088B
:10014000030200080302000803020008E52E00086D
:10015000030200080302000803020008030200086B
:10016000030200080302000803020008030200085B
:10017000030200080302000803020008030200084B
:1001800003020008030200085D10000803020008D3
:10019000030200080302000803020008030200082B
:1001A000030200080302000803020008030200081B
:1001B000030200080302000803020008030200080B
:1001C00003020008030200080302000803020008FB
:1001D00003020008030200080302000803020008EB
:1001E00003020008030200080302000803020008DB
:1001F00003020008030200080302000803020008CB
:1002000002E000F000F8FEE772B6394880F3088893
:10021000384880F3098838484EF60851CEF200017C
:10022000086040F20000CCF200004EF63471CEF2CD
:1002300000010860BFF34F8FBFF36F8F40F20000E3
:10024000C0F2F0004EF68851CEF200010860BFF314
:100250004F8FBFF36F8F4FF00000E1EE100A4EF6A4
:100260003C71CEF200010860062080F31488BFF3D1
:100270006F8F02F0BFFA03F025FA4FF055301F4997
:100280001B4A91423CBF41F8040BFAE71C49194A4A
:1002900091423CBF41F8040BFAE71A491A4A1B4B3A
:1002A0009A423EBF51F8040B42F8040BF8E70020D5
:1002B0001749184A91423CBF41F8040BFAE702F093
:1002C000DDFA03F069FA144C144DAC4203DA54F829
:1002D000041B8847F9E700F03FF8114C114DAC4280
:1002E00003DA54F8041B8847F9E702F0C5BA0000A6
:1002F0000004022000240220000000080000022068
:1003000000040220483F000800240220502402205C
:1003100050240220D8340220000200080002000805
:1003200000020008000200082DE9F04F2DED108AB0
:10033000C1F80CD0D0F80CD0BDEC108ABDE8F08F1D
:10034000002383F311882846A047002001F098FE7F
:1003500001F048FE00DFFEE770B5214C6FF070033E
:10036000002523706FF07F061E236570A570E57071
:1003700025716571A571E57125726672A372E572CA
:1003800000F02EFD20B10E2325726672A372E57275
:1003900002F0B4F9044602F0E9F90546D8B9114B68
:1003A0009C421AD001339C4218BF054641F2883462
:1003B00004BF01250024002002F0AAF90DB100F0CD
:1003C000B7F800F07FFD00F05DFC204600F050F92A
:1003D00000F0AEF8F9E70024EDE70446EBE700BFD4
:1003E00050240220010007B008B500F0C9FBA0F1BD
:1003F00020035842584108BD07B5054B02211B8810
:10040000ADF8043001A800F027FC03B05DF804FB50
:10041000BC3B0008064991F8243033B10023082280
:10042000086A81F8243000F051BC0120704700BFF9
:10043000702402202DE9F84F234C94F8243005460F
:10044000884617468BBB2E46DFF87C90002F38D0AD
:1004500094F824A0BAF1000F05D12022FF214846CC
:10046000266200F01DFDCAF10805BD4228BF3D46C9
:100470005FFA85FBAD0041462A4604EB8A0000F096
:10048000E5FC94F82430A7EB0B079B445FFA8BFB49
:10049000BBF1080F2E44A844FFB284F824B0D5D194
:1004A000FFF7B8FF0028D1D108E0266A06EB8306E3
:1004B000B042C9D0FFF7AEFF0028C4D10020BDE88C
:1004C000F88F0120BDE8F88F7024022010B520239A
:1004D00083F311881248C3680BB101F057FE002363
:1004E000104A0F484FF47A7101F014FE002383F391
:1004F00011880D4C236813B12368013B23606368A6
:1005000013B16368013B6360084B1B7833B96368C0
:1005100023B9022000F090FC3223636010BD00BFBD
:100520005C240220CD040008A0250220982402208B
:100530002DE9F041444B454953F8042F013201D1D4
:10054000BDE8F0818B42F7D1414C424B22689A4280
:1005500078D9414B9B6803F1006303F5C0339A429D
:1005600070D2002000F0AAFB3C4B0220187000F073
:1005700059FC3B4B1A6C00221A64196E1A66196EEC
:10058000596C5A64596E5A66596E596941F0800126
:100590005961596921F0800159615969196941F01E
:1005A00000511961196921F0005119611B6972B676
:1005B0002C492D4B0B601D682468BFF34F8FBFF390
:1005C0006F8F2A4BC3F88420BFF34F8F5A6922F4F0
:1005D00080325A61BFF34F8FD3F88020C2F3C9062F
:1005E000C2F34E325201B70743F6E07E02EA0E082C
:1005F00038463146013948EA000CB1F1FF3FC3F8F3
:1006000074C200F14040F5D1203A12F1200FEDD133
:10061000BFF34F8FBFF36F8FBFF34F8FBFF36F8F5A
:100620005A6922F400325A610022C3F85022BFF303
:100630004F8FBFF36F8F202383F31188AD4685F36F
:1006400008882047BDE8F081FC7F01081C80010874
:1006500004800108FF7F0108502402209824022012
:100660000038024008ED00E00080010800ED00E0E5
:100670002DE9F04F99B0B34C01902022FF2110A832
:10068000A66800F00DFCB04A1378A346A3B9AF48A2
:100690000121C3601170202383F31188C3680BB15B
:1006A00001F074FD0023AA4AA8484FF47A7101F0C2
:1006B00031FD002383F31188019B13B1A54B019AEF
:1006C0001A60A54AA349019F0292002313704B6050
:1006D00099461C461D469846012000F0A3FB002FBA
:1006E00000F012829B4B1B68002B40F00D8219B06A
:1006F000BDE8F08F0220FFF777FE002840F0FB8175
:10070000019BB9F1000F08BF1F46944B1B88ADF841
:100710002C3002210BA800F09FFADDE74FF47A702D
:1007200000F02EFA031E0393EADB0220FFF75CFEC3
:1007300082460028E4D0039B581E042800F2DD8185
:10074000DFE800F0030E1114170018A8052340F885
:10075000343D042100F080FA54464FF0000856E082
:1007600004217848F6E704217D48F3E704217D4819
:10077000F0E71C24204600F0A3FA04340B90042177
:100780000BA800F069FA2C2CF4D1E5E7002DB7D0C6
:10079000002CB5D00220FFF727FE0546002800F008
:1007A000AF8101206C4C00F089FA0220207000F02B
:1007B00039FB4FF000095FFA89FA504600F08EFAD3
:1007C000074658B1504600F099FA09F1010900288E
:1007D000F1D12C46A9460027634B97E7012302205D
:1007E000237000F015FB3E46DBF808309E4206D22F
:1007F000304600F065FA0130EBD10436F4E7029B95
:1008000000261E70534BA9465E602C46374600F00A
:100810004FFB15B1002C18BF0027FFF7EDFD5BE77C
:10082000002D3FF46DAF002C3FF46AAF029B022015
:10083000187000F0F7FA322000F0A2F9B0F1000AC7
:10084000C0F25E811AF0030540F05A81DBF80820FF
:1008500006EB0A03934200F25381BAF5807F00F25F
:100860004F8155450DDA4FF47A7000F089F9049004
:10087000049B002BC0F244813C4A049BAB540135DD
:10088000EFE7C820FFF7B0FD0546002800F03881EB
:100890001F2E11D8C6F12004544528BF544610AB72
:1008A00026F0030022463149184400F0CFFA2246D0
:1008B000FF212E4800F0F4FA4FEAAA0A5FFA8AF202
:1008C0002A493046FFF7B6FD0446002800F01A8199
:1008D00006EB8A0605469AE70220FFF785FD002809
:1008E0003FF40EAFFFF796FD00283FF409AF4FF03D
:1008F000000A5346DBF8082092451CD2BAF11F0FBC
:1009000012D8109A01320FD02AF0030218A90A4413
:1009100052F8202C0B92184604220BA900F06AFB17
:100920000AF1040A0346E5E75046039300F0C8F9CC
:10093000039B0B90EFE718A8042140F84C3D00F012
:100940008BF964E7502402209C2502205C240220BD
:10095000CD040008A025022098240220BE3B0008F8
:100960005424022058240220C03B00089C2402206A
:1009700018A8002340F8343D642100F039F900281C
:100980007FF4BEAE0220FFF72FFD00283FF4B8AE83
:100990000B9800F0C5F918AB43F8480D0421184630
:1009A000CDE718A8002340F8343D642100F020F979
:1009B00000287FF4A5AE0220FFF716FD00283FF4C3
:1009C0009FAE0B9800F0BAF918AB43F8440DE5E779
:1009D0000220FFF709FD00283FF492AE00F0B4F9C1
:1009E00018AB43F8400DD9E70220FFF7FDFC0028C3
:1009F0003FF486AE0BA9142000F0ACF9824618A88B
:100A0000042140F83CAD00F027F951460BA896E7C9
:100A1000322000F0B5F8B0F1000AFFF671AE1AF01E
:100A2000030F7FF46DAEDBF808200AEB0803934256
:100A30003FF666AE0220FFF7D7FC00283FF460AE19
:100A40002AF0030AC244D0453FF4E1AE404600F02C
:100A500037F904210A900AA800F0FEF808F104080A
:100A6000F1E74FF47A70FFF7BFFC00283FF448AE7F
:100A7000FFF7D0FC00283FF4AFAE109B01330CD041
:100A8000082210A90020FFF7D5FC00283FF4A4AEEF
:100A90002022FF2110A800F003FAFFF7ADFC374831
:100AA00001F0F4FA23E6002D3FF42AAE002C3FF4C7
:100AB00027AE18A8002340F8343D642100F098F8D0
:100AC000824600287FF41CAE0220FFF78DFC002830
:100AD0003FF416AE0390FFF78FFC41F2883001F02F
:100AE000D5FA0B9800F026FA00F0E2F9039B57467E
:100AF0001C461D46F0E5054689E64FF00008FFE577
:100B00002546FDE52C4667E6002000F039F8049004
:100B1000049B002BFFF6E3AD012000F079F9049B64
:100B2000213B122B3FF6D8AD01A252F823F000BFB3
:100B3000F50600081D0700088D070008D906000803
:100B4000D9060008D906000821080008110A000883
:100B5000D908000871090008A3090008D109000894
:100B6000D9060008E9090008D9060008630A000848
:100B70000F080008D9060008A70A0008A08601008F
:100B80002DE9F34702AE00244FF47A7506F8014DC3
:100B9000144FDFF85880454397F900305A1C5FFA2C
:100BA00084F901D0A34212D158F82400036801222D
:100BB000D3F820A031462B46D047012807D10A4B55
:100BC0009DF8070083F8009002B0BDE8F08701347B
:100BD000022CE1D14FF4FA7001F058FA4FF0FF30D7
:100BE000F2E700BF00240220C4250220CC3B00080D
:100BF0002DE9F0474FF47A75144FDFF85880064618
:100C00004D43002497F900305A1C5FFA84F901D053
:100C1000A34210D158F8240003680422D3F820A07E
:100C200031462B46D047042805D1094B83F8009064
:100C30000020BDE8F0870134022CE3D14FF4FA70B4
:100C400001F024FA4FF0FF30BDE8F08700240220C5
:100C5000C4250220CC3B000830B4074B1A78074B60
:100C600053F822402368DD69054B0A46AC4601462D
:100C7000204630BC604700BFC4250220CC3B0008A2
:100C8000A0860100F8B501F03DFC094C094E0A4F61
:100C90002070002530682378834207D901F02CFCAE
:100CA000336805440133BD423360F3D9F8BD00BF5A
:100CB000C5250220A8250220FF7F010001F0D0BC3D
:100CC00000F1006000F5C0300068704700F100607E
:100CD000920000F5C03001F05BBC0000054B1A68C3
:100CE000054B1B789B1A834202D9104401F004BCC7
:100CF00000207047A8250220C525022038B5074DE1
:100D000004462868204401F0FFFB28B928682044E5
:100D1000BDE8384001F010BC38BD00BFA825022056
:100D200010F0030308D1B0F5806F05D800F1005032
:100D3000A0F571200068704700207047014BC05833
:100D4000704700BF20F4F01F014B1868704700BFC8
:100D5000002004E0F0B5204B1E68204B1F885D6822
:100D600093F90840C6F30B02BA424FEA164622D066
:100D70009F89BA4221D01F8BBA4206D102220C248D
:100D800004FB02335D6893F90840B6F5805F16D026
:100D900041F201039E4208BF5A24421E0A44013D0B
:100DA0000B46934215D215F9016F581C4EB10346FC
:100DB00000F8016CF5E70022E1E70122DFE74124BA
:100DC000EBE72C2582421D7001D9981C5C70401AFB
:100DD000F0BD1846FBE700BF002004E00424022019
:100DE000094B5B88B3F5805F09D041F20102934261
:100DF00007D10122054B03EB8203D878704700220C
:100E0000F8E70020704700BF002004E0C43B000862
:100E1000022802BF024B4FF080629A61704700BF08
:100E2000000C0240022802BF024B4FF480629A611C
:100E3000704700BF000C0240022801BF024A5369FC
:100E400083F4806353617047000C024010B50023A7
:100E5000934203D0CC5CC4540133F9E710BD0000C9
:100E600030B5441E14F9010F0B4660B193F90050E0
:100E7000854201F1010106D11AB993F90020801AC7
:100E800030BD013AEEE7002AF7D1104630BD000030
:100E900002460346981A13F9011B0029FAD170473C
:100EA00002440346934202D003F8011BFAE770475D
:100EB000024B1A78024B1A70704700BFC4250220FB
:100EC0000024022038B5154C154D204600F01EFCBC
:100ED0002946204600F046FC2D681248EA6ED2F8FA
:100EE000043843F00203C2F8043801F0CFF80E4989
:100EF000284600F045FDEA6E0C48D2F804380C494B
:100F000023F00203C2F80438A0424FF4E1330B602F
:100F100003D0BDE8384000F057BB38BDF42A0220AA
:100F2000BC3C000840420F00E43C00084826022078
:100F3000AC25022038B50B4B1A780B4B53F82240E6
:100F40000A4B9C4205460CD0094B0021184618223A
:100F5000FFF7A6FF056001462046BDE8384000F0D7
:100F600033BB38BDC4250220CC3B0008F42A022044
:100F7000AC250220FEE7000000B59BB0EFF309812D
:100F800068226846FFF762FFEFF30583034B9A6B15
:100F90009A6A9A6A9A6A9A6A9B6AFEE700ED00E08A
:100FA00000B59BB0EFF3098168226846FFF74EFF5A
:100FB000EFF30583044B9A6B9A6A9A6A9A6A9A6A63
:100FC0009A6A9B6AFEE700BF00ED00E000B59BB0A7
:100FD000EFF3098168226846FFF738FFEFF30583D6
:100FE000034B5A6B9A6A9A6A9A6A9A6A9B6AFEE7F4
:100FF00000ED00E030B5084D0A4491420BD011F8E5
:10100000013B09245840013CF7D040F300032B403A
:1010100083EA5000F7E730BD2083B8ED0023044990
:101020001A465A50C8180833802B4260F9D17047CD
:10103000C8250220024A136843F0C00313607047BA
:1010400000780040044B5A6810439A6858600AB10F
:10105000181D1047704700BF482602202DE9F84FA1
:10106000404EF56D2F68EC692C62210718D014F002
:10107000080F0CBF00208020E20748BF40F020008E
:10108000A30748BF40F04000610748BF40F48070AC
:10109000202383F31188FFF7D5FF002383F3118802
:1010A000E20509D5202383F311884FF40070FFF780
:1010B000C9FF002383F31188DFF8A8A04FF02009AF
:1010C0004FF0000B14F0200832D13B0615D5DFF8A5
:1010D00098A04FF0200920060FD589F311885046BB
:1010E00000F0E6F9002830DA0820FFF7ABFF27F020
:1010F00080032B60002383F3118879060DD56206E7
:101100000BD5202383F31188F26C336D9A4201D101
:10111000336CFBB9002383F31188E30604D5B26E68
:1011200013690BB150699847BDE8F84F01F034BB23
:1011300089F311886B6A96F864105046194000F0E4
:1011400051FA8BF31188EC69BCE7A86288F3118827
:10115000EC69C0E7102027F04007FFF773FF2F600E
:10116000D8E700BF482602208026022013B5104C85
:10117000204600F01DFA04F11400009400234FF4FF
:1011800000720C4900F0DEF804F1380000940A4BBC
:101190000A494FF4007200F057F9094BE365094B17
:1011A00023660B21522002B0BDE8104000F058B871
:1011B00048260220B426022035100008B428022058
:1011C0000078004080F93703224B002908BF1946F8
:1011D000037C8166012B30B50CD11F4B984209D19D
:1011E0001E4B1A6C42F080421A641A6E42F0804222
:1011F0001A661B6E0A68036EC46D03EB5203B3FBE1
:10120000F2F34A68150442BF23F0070503F0070311
:1012100043EA4503E3608B6843F040036360CB68B7
:1012200043F00103A36042F4967343F0010323608B
:1012300051054FF0FF33236205D512F0102205D07F
:10124000B2F1805F04D080F8643030BD7F23FAE7CC
:101250003F23F8E7003C00084826022000380240FF
:1012600000F1604300F01F02400903F561430901EA
:101270008000C9B200F1604083F8001300F56140BE
:1012800001239340C0F8803103607047F8B51546DC
:1012900082680669AA420B46816938BF8568761A5A
:1012A000B542044607D218462A46FFF7CFFDA36988
:1012B0002B44A3610DE011D932461846FFF7C6FD55
:1012C000AF1B3A46E1683044FFF7C0FDE2683A449C
:1012D000A261A3685B1BA3602846F8BD18462A4696
:1012E000FFF7B4FDE368E4E783682DE9F0410446C5
:1012F00093421546266938BF85684069361AB5425B
:101300000F4606D22A46FFF7A1FD63692B446361AD
:101310000DE012D93246A5EB0608FFF797FD4246CD
:10132000B919E068FFF792FDE26842446261A36880
:101330005B1BA3602846BDE8F0812A46FFF786FDC7
:10134000E368E4E710B50A440024C361029B00602F
:1013500040608460C160816141610261036210BDCF
:1013600008B582694369934201D1826882B9826873
:10137000013282605A1C42611970426903699A42C3
:1013800001D3C3684361002100F09CFE002008BD2A
:101390004FF0FF3008BD000070B5202304460E4614
:1013A00083F31188A568A5B1A368A269013BA36076
:1013B000531CA36115782269934224BFE368A3619B
:1013C000E3690BB120469847002383F31188284630
:1013D00070BD3146204600F065FE0028E2DA85F354
:1013E000118870BD2DE9F74F05460F4690469A4685
:1013F000D0F81C90202686F311884FF0000B14467D
:1014000064B1224639462846FFF740FF034668B9D3
:101410005146284600F046FE0028F1D0002383F311
:101420001188A8EB040003B0BDE8F08FB9F1000FFC
:1014300003D001902846C847019B8BF31188E41A1A
:101440001F4486F31188DBE7C16081614161C3619C
:101450001144009B0060406082600161036270473C
:10146000F8B504460E461746202383F31188A56875
:10147000A5B1A368013BA36063695A1C62611E7039
:10148000236962699A4224BFE3686361E3690BB12F
:1014900020469847002080F31188F8BD3946204641
:1014A00000F000FE0028E2DA85F31188F8BD0000A4
:1014B000836942699A4210B501D182687AB982681B
:1014C000013282605A1C82611C7803699A4201D3FE
:1014D000C3688361002100F0F5FD204610BD4FF088
:1014E000FF3010BD2DE9F74F05460F4690469A464E
:1014F000D0F81C90202686F311884FF0000B14467C
:1015000064B1224639462846FFF7EEFE034668B925
:101510005146284600F0C6FD0028F1D0002383F391
:101520001188A8EB040003B0BDE8F08FB9F1000FFB
:1015300003D001902846C847019B8BF31188E41A19
:101540001F4486F31188DBE702684368114301609A
:1015500003B11847704700001430FFF743BF000085
:101560004FF0FF331430FFF73DBF00003830FFF776
:10157000B9BF00004FF0FF333830FFF7B3BF0000B2
:101580001430FFF709BF00004FF0FF311430FFF7B0
:1015900003BF00003830FFF763BF00004FF0FF3299
:1015A0003830FFF75DBF000000207047FFF7DEBD59
:1015B000044B0360002343608360C3600123037412
:1015C000704700BF183C000810B52023044683F381
:1015D0001188FFF7F9FD02232374002383F3118898
:1015E00010BD000038B5C36904460D461BB904217F
:1015F0000844FFF7A9FF294604F11400FFF7B0FEE5
:10160000002806DA201D4FF48061BDE83840FFF75E
:101610009BBF38BD026843681143016003B118479E
:101620007047000013B5446BD4F894341A681178ED
:10163000042915D1217C022912D11979128901239B
:101640008B4013420CD101A904F14C0001F0AEFE15
:10165000D4F89444019B21790246206800F0E0F917
:1016600002B010BD143001F031BE00004FF0FF3366
:10167000143001F02BBE00004C3001F003BF00001D
:101680004FF0FF334C3001F0FDBE0000143001F08C
:10169000FFBD00004FF0FF31143001F0F9BD000034
:1016A0004C3001F0CFBE00004FF0FF324C3001F063
:1016B000C9BE0000D0F8942438B5136819780429FD
:1016C000054601D0012038BD017C0229FAD11279EA
:1016D0005C89012090400440F4D105F1140001F030
:1016E00091FD02460028EDD0D5F894544FF4807354
:1016F0002868697900F082F9204638BD406BFFF711
:10170000D9BF000000207047704700007FB5124B22
:101710000360002343608360C360012502260F4BF2
:10172000057404460290019300F184022946009654
:101730004FF48073143001F041FD094B0193029482
:1017400000964FF4807304F52372294604F14C008F
:1017500001F008FE04B070BD403C0008FD16000812
:10176000251600080B68202282F311880A7903EB02
:10177000820210624A790D3243F822008A7912B14E
:1017800003EB8203186202230374C0F8941400234D
:1017900083F311887047000038B5037F044613B106
:1017A00090F85430ABB9201D01250221FFF732FF1C
:1017B00004F1140025776FF0010100F08FFC84F82C
:1017C000545004F14C006FF00101BDE8384000F0C6
:1017D00085BC38BD10B5012104460430FFF71AFF5F
:1017E0000023237784F8543010BD000038B5044638
:1017F0000025143001F0FAFC04F14C00257701F0CB
:10180000C9FD201D84F854500121FFF703FF204635
:10181000BDE83840FFF74EBF90F85C3003F060033E
:10182000202B19D190F85D20212A0AD0222A4FF0CE
:1018300000030ED0202A0FD1084A02650722426514
:1018400004E0064B036507234365002383650120FD
:10185000704703654365F9E700207047282402209C
:10186000D0F8943437B51A681178042904461AD18F
:10187000017C022917D11979128901238B40134267
:1018800011D100F14C05284601F044FE58B101A9E0
:10189000284601F08BFDD4F89444019B217902463F
:1018A000206800F0BDF803B030BD000000EB8103FC
:1018B000F7B51C6A05460E46F4B1202383F3118860
:1018C00005EB8607201D0821FFF7A4FEFB685B6976
:1018D0001B684C3413B1204601F076FD01A9204667
:1018E00001F064FD024648B1019B3146284600F0F4
:1018F00097F8002383F3118803B0F0BDFB685A69A1
:101900001268002AF5D01B8A013B1340F1D105F182
:101910005C02EAE70D3138B550F82140DCB12023F4
:1019200083F31188D4F894241368527903EB82036B
:10193000DB689B695D6845B104216018FFF76AFEAA
:10194000294604F1140001F067FC2046FFF7B2FEBF
:10195000002383F3118838BD7047000001F014B8EC
:10196000012303700023436000F1240200F13801D9
:1019700042F8043B8A421361FAD1038143817047E4
:1019800038B50446202383F3118800254160C560E3
:10199000056145618561C561056201F005F80223B5
:1019A000237085F3118838BD70B500EB81030546BF
:1019B0005069DA600E46144618B110220021FFF774
:1019C0006FFAA06918B110220021FFF769FA3146B9
:1019D0002846BDE8704001F0B1B80000028902F06D
:1019E00001020281428902F0010242810022026169
:1019F00042618261C261026201F034B9F0B400EB6D
:101A000081044789E4680125A4698D403D434581EF
:101A100023600023A2606360F0BC01F04FB90000B6
:101A2000F0B400EB81040789E468012564698D4006
:101A30003D43058123600023A2606360F0BC01F098
:101A4000C9B9000070B50223002504460370A0F850
:101A5000645080F8665080F8675005814581C56004
:101A6000056145618561C561056280F84C5001F0F2
:101A700001F863681B6823B129462046BDE8704021
:101A8000184770BD436802781B6880F868200522FB
:101A900002700BB10421184770470000436890F8AA
:101AA00068201B6802700BB10521184770470000C1
:101AB00090F84C3070B5044613B1002380F84C30D8
:101AC00004F15C02204601F0EFF863689B6863BB99
:101AD00094F85C5015F0600615D194F85D3005F06F
:101AE0007F0545EA032540F202339D4200F00E8156
:101AF0005BD8022D00F0DC803FD8002D00F08780FD
:101B0000012D00F0CF800021204601F039FB00219B
:101B1000204601F02BFB63681B6813B106212046A9
:101B20009847062384F84C3070BD2046984700281B
:101B3000CED094F8632094F8623043EA0223626DB9
:101B4000934238BF636594F95C30656D002B4FF0AC
:101B5000200380F2FD80002D00F0EC80092284F843
:101B60004C2083F311880021636D226D2046FFF71E
:101B700057FF002383F3118870BDB5F5817F00F016
:101B8000B180B5F5407F49D0B5F5807FBBD194F8E1
:101B90005E30012BB7D1B4F8643023F00203A4F80F
:101BA000643026656665A665C3E740F201639D4221
:101BB0001ED8B5F5C06F3BD2B5F5A06FA3D1B4F870
:101BC0005C30B3F5A06F0ED194F85E3084F86630C7
:101BD000204600F0A7FF63681B6813B1012120466F
:101BE000984703232370002323656365A365A0E75B
:101BF000B5F5106F32D040F602439D4252D0B5F594
:101C0000006F80D104F167032365012324E004F110
:101C10006403236502236365A5658AE794F85E3053
:101C2000012B7FF470AFB4F8643043F00203B6E7E1
:101C300094F86120616894F860304D6894F85F1002
:101C400043EA0223204694F85E20A84700283FF488
:101C50005AAF4368236503686365A4E72378042BC0
:101C600010D1202383F311882046FFF7B7FE86F3B7
:101C70001188636884F867601B68032121700BB1C9
:101C80002046984794F85E30002BACD084F867303B
:101C90000423237063681B68002BA4D00221204614
:101CA0009847A0E7374B23650223636500239DE730
:101CB00094F8601011F0800F204601F00F010ED053
:101CC00000F0E4FF012806D002287FF41CAF2E4B61
:101CD0002365606567E72D4B2365656563E700F065
:101CE000C7FFEFE794F85E30002B7FF40CAF94F859
:101CF000603013F00F013FF476AF1A06204602D58C
:101D000001F052FA6FE701F045FA6CE794F85E30A3
:101D1000002B7FF4F8AE94F8603013F00F013FF41D
:101D200062AF1B06204602D501F02AFA5BE701F0FC
:101D30001DFA58E7142284F84C2083F311882B46AF
:101D40002A4629462046FFF759FE85F3118870BDC3
:101D50005DB1152284F84C2083F311880021636D56
:101D6000226D2046FFF74AFE03E70B2284F84C2041
:101D700083F311882B462A4629462046FFF750FE5A
:101D8000E3E700BF703C0008683C00086C3C0008BA
:101D900038B590F84C300446152B29D8DFE803F00D
:101DA0003E28282828283E28280B29392828282892
:101DB000282828283E3E90F8631090F86220436D52
:101DC00042EA01229A4214D9C268128AB3FBF2F5A0
:101DD00002FB15356DB9202383F311882B462A4663
:101DE0002946FFF71DFE85F311880A2384F84C303D
:101DF00038BD142384F84C30202383F3118800234A
:101E00001A4619462046FFF7F9FD002383F311888F
:101E100038BD836D03B198470023E7E7002101F047
:101E2000AFF90021204601F0A1F963681B6813B1E6
:101E30000621204698470623D8E7000090F84C205A
:101E4000152A38B5044622D80123934040F6416252
:101E500013421DD113F480150FD19B0217D50B230C
:101E600080F84C30202383F311882B462A462946DC
:101E7000FFF7D6FD85F3118838BDC3689B695B68A1
:101E80002BB9836D03B19847002384F84C3038BDDB
:101E9000002101F075F90021204601F067F963681F
:101EA0001B6813B10621204698470623EDE7000082
:101EB000024B00221B605B609A607047B42A0220CC
:101EC000002303748268054B1B6899689142FBD21A
:101ED0005A6803604260106058607047B42A02205C
:101EE00008B5202383F31188037C032B05D0042B32
:101EF0000DD02BB983F3118808BD436900221A6005
:101F00004FF0FF334361FFF7DBFF0023F2E790E878
:101F10000C001A6002685360F2E7000000230374AB
:101F20008268054B1B6899689142FBD85A68036028
:101F30004260106058607047B42A0220054B19694E
:101F40000874186802681A605360186101230374EA
:101F5000FEF7EAB9B42A022030B54B1C87B005461B
:101F60000A4C10D023690A4A01A800F0D3F8284689
:101F7000FFF7E4FF049B13B101A800F007F9236900
:101F8000586907B030BDFFF7D9FFF8E7B42A02203F
:101F9000E11E000838B50C4D41612B6981689A68D3
:101FA0009142044603D8BDE83840FFF789BF184680
:101FB000FFF786FF01232C61014623742046BDE80C
:101FC0003840FEF7B1B900BFB42A0220044B1A68AA
:101FD0001B6990689B68984294BF0020012070475D
:101FE000B42A022010B5084C236820691A682260C0
:101FF0005460012223611A74FFF790FF01462069A3
:10200000BDE81040FEF790B9B42A02208260022297
:1020100002740022427470478368A3F17C0243F883
:102020000C2C026943F83C2C426943F8382C074ACF
:1020300043F81C2CC26843F8102C022203F8082C29
:10204000002203F8072CA3F1180070474103000891
:1020500010B5202383F31188FFF7DEFF002104462B
:10206000FFF798FF002383F31188204610BD00007E
:10207000024B1B6958610F20FFF760BFB42A022092
:10208000202383F31188FFF7F3BF000008B5014652
:10209000202383F311880820FFF75EFF002383F3DA
:1020A000118808BD49B1064B42681B6918605A6027
:1020B000136043600420FFF74FBF4FF0FF307047BD
:1020C000B42A02200368984206D01A680260506061
:1020D00059611846FFF7F4BE7047000038B5044652
:1020E0000D462068844200D138BD036823605C60DF
:1020F0004561FFF7E5FEF4E7054B03F114025A6171
:102100009A614FF0FF32DA6100221A62704700BF15
:10211000B42A0220F8B503614FF08043C2605C6AC4
:10212000194B1A46022952F8145F38BF0221954212
:1021300006461F460AD1586198611C6205604560D9
:1021400081600819BDE8F84001F006BA186AAB686A
:10215000241A0C1902D3E41A2D6804E09C4202D21E
:10216000204401F007FAAB689C42F4D86B687360B6
:1021700035601E606E60B460A9684FF0FF33091BC4
:10218000A960FB61F8BD00BFB42A022010B41B4C4B
:10219000234653F8141F814210D0416802680A6038
:1021A000026851609A424FF00001C16003D0936809
:1021B00081680B4493605DF8044B70470A68626164
:1021C00000209A425360C86003D15DF8044B01F0CF
:1021D000CBB993688868034493604FF08042206ACB
:1021E000526A121A9342E6D9991A012998BF931C90
:1021F00018445DF8044B01F0BDB900BFB42A0220B9
:1022000000207047FEE70000704700004FF0FF30ED
:1022100070470000022906D0032906D0012906488C
:1022200018BF0020704705487047032A9ABF04482A
:1022300000EBC20000207047403D0008F43C00085D
:102240003024022070B59AB001AD064608462946F2
:10225000144600F095F82846FEF71AFEC0B2431C5B
:102260005B0086E8180023700323637000230234A8
:102270001946DAB2904204F1020401D81AB070BDD6
:10228000EA5C04F8022C04F8011C0133F1E70000B9
:1022900008B5202383F311880348FFF7E1FA0023F0
:1022A00083F3118808BD00BFF42A022010B504464C
:1022B000052916D8DFE801F016150316161D202390
:1022C00083F311880E4A0121FFF76EFB20460D4A69
:1022D0000221FFF769FB0C48FFF788FA002383F31C
:1022E000118810BD202383F311880748FFF754FAA3
:1022F000F4E7202383F311880348FFF76BFAEDE737
:10230000743C0008983C0008F42A022038B50C4DB3
:102310000C4C0D492A4604F10800FFF793FF05F124
:10232000CA0204F110000949FFF78CFF05F5CA72D3
:1023300004F118000649BDE83840FFF783BF00BF2D
:10234000BC2F022030240220C43C0008CE3C0008F0
:10235000D93C000870B5044608460D46FEF798FDC6
:10236000C6B22046013403780BB9184670BD324618
:102370002946FEF775FD0028F3D1012070BD00004D
:102380002DE9F04704460D46FEF782FD2C49C6B202
:102390002046FFF7DFFF08B10736F6B2294920468D
:1023A000FFF7D8FF08B11036F6B2632E0BD8DFF86E
:1023B0009080DFF89090244FDFF898A0267846B9F7
:1023C0002E70BDE8F08721462846BDE8F04701F0B1
:1023D000EDBB252E2FD1072241462046FEF740FDBA
:1023E00070B91A4B2A4603F10C0153F8040B42F85A
:1023F000040B8B42F9D11B88138007340E35DDE7BF
:10240000082249462046FEF72BFDA0B9104BAA1C16
:1024100013F8011F09095345C95D02F8021C197818
:1024200001F00F0102F10202C95D02F8031CEFD1B5
:1024300018350834C2E72E7001340135BEE700BFFD
:10244000603D0008D93C0008773D0008683D000861
:102450001FF4F01F2BF4F01FBFF34F8F024AD36815
:10246000DB03FCD4704700BF003C024008B5074BBB
:102470001B7853B9FFF7F0FF054B1A69002ABFBF5D
:10248000044A5A6002F188325A6008BD1A320220AA
:10249000003C02402301674508B5054B1B7833B962
:1024A000FFF7DAFF034A136943F00043136108BDE5
:1024B0001A320220003C02400B2870B513D80B4A98
:1024C0000B4C137863B90B4E4FF0006144F82310A6
:1024D00056F8235001330C2B2944F7D101231370F4
:1024E00054F8200070BD002070BD00BF4C320220A7
:1024F0001C320220883D0008014B53F82000704731
:10250000883D00080C2070470B2810B5044601D9FF
:10251000002010BDFFF7D0FF064B53F824301844BD
:10252000C21A0BB9012010BD12680132F0D1043B70
:10253000F6E700BF883D00080B2810B5044621D8F7
:10254000FFF78AFFFFF792FF0F4AF323D360C30020
:10255000DBB243F4007343F002031361136943F4E5
:1025600080331361FFF778FFFFF7A6FF074B53F89F
:10257000241000F0DDF8FFF78FFF2046BDE8104083
:10258000FFF7C2BF002010BD003C0240883D00089C
:102590002DE9F84312F00103154640D18218B2F13B
:1025A000026F3CD22C4B1B6813F0010337D02B4C2D
:1025B000FFF75CFFF323E360FFF74EFF40F20127D4
:1025C000032D01D9830713D0244C0F46401A40F243
:1025D0000118EB1B0B44012B00EB0706236924D8E1
:1025E00023F001032361FFF757FF0120BDE8F883C3
:1025F000236923F44073236123693B43236151F82A
:10260000046B0660BFF34F8FFFF726FF03689E42FF
:1026100008D0236923F001032361FFF73DFF002069
:10262000BDE8F883043D0430CAE723F44073236116
:10263000236943EA08032361B94637F8023B338034
:10264000BFF34F8FFFF708FF3688B9F80030B6B2F6
:10265000B342BED0DDE700BF00380240003C02407C
:10266000084908B50B7828B153B9FFF7FFFE0123DD
:102670000B7008BD23B1BDE808400870FFF70CBF20
:1026800008BD00BF1A32022010B50244064B0439BF
:10269000D2B2904200D110BD441C00B253F82000C9
:1026A00041F8040FE0B2F4E750280040104B30B579
:1026B0001C6F240407D41C6F44F400741C671C6F47
:1026C00044F400441C670B4C236843F4807323607C
:1026D0000244094B0439D2B2904200D130BD441CAF
:1026E00000B251F8045F43F82050E0B2F4E700BFB5
:1026F00000380240007000405028004007B5012219
:1027000001A90020FFF7C0FF019803B05DF804FBAA
:1027100013B50446FFF7F2FFA04206D002A901223A
:1027200041F8044D0020FFF7C1FF02B010BD0000CA
:102730000144BFF34F8F064B884204D3BFF34F8F42
:10274000BFF36F8F7047C3F85C022030F4E700BF1F
:1027500000ED00E0034B1B689B0042BF024B0122CF
:102760001A707047743802404D320220014B1878BD
:10277000704700BF4D320220064A536823F0010320
:102780005360EFF30983683383F30988002383F3ED
:102790001188704730EF00E010B5202383F31188D3
:1027A000104B5B6813F4006318D0F1EE103AEFF3AE
:1027B00009844FF0807344F84C3C0B4BDB6844F8C1
:1027C000083CA4F1680383F30988FFF7FFFB18B105
:1027D000064B44F8503C10BD054BFAE783F31188D3
:1027E00010BD00BF00ED00E030EF00E05103000835
:1027F00054030008F0B5BFF34F8FBFF36F8F1D4B2D
:102800000021C3F85012BFF34F8FBFF36F8F5A6987
:1028100042F400325A61BFF34F8FBFF36F8FC3F89A
:102820008410BFF34F8FD3F88020C2F3C904C2F3E2
:102830004E325201A50743F6E07602EA060E28461C
:1028400021464EEA00070139C3F860724F1C00F1BF
:102850004040F6D1203A12F1200FEED1BFF34F8F56
:102860005A6942F480325A61BFF34F8FBFF36F8FC2
:10287000F0BD00BF00ED00E0FEE70000084A094B94
:1028800009498B4204D3094A0021934205D370477A
:1028900052F8040F43F8040BF3E743F8041BF4E782
:1028A000943F0008D8340220D8340220D8340220C3
:1028B000036F30B500229D68C46E11464FF0FF30A3
:1028C00004EB421301329542C3F80019C3F8101902
:1028D000C3F80809C3F8001BC3F8101BC3F8080BA2
:1028E000EED24FF00113C4F81C3830BD890141F01D
:1028F0002001016103699B06FCD4122000F0C8BED0
:10290000204B03EB80022DE9F047D2F80CE0DD6E9E
:10291000DEF81420461CD2F800C005EB063605EBA5
:102920004018516861450BD3D5F83428012303FAC8
:1029300000F022EA0000C5F834081846BDE8F08728
:10294000BEF81040ACEB0103A34228BF2346D8F8E1
:102950001849A4B2B3EB840F10D894681F46A4F1B1
:10296000040959F804AFC6F800A0042F01D9043FA8
:10297000F7E71C440B4494605360D2E70020BDE8A5
:10298000F08700BF5032022010B5054C2046FEF7FC
:10299000E7FF4FF0A043E366024B236710BD00BF83
:1029A00050320220DC3D00080378012B70B505464B
:1029B00050D12A4BC46E98421BD1294B5A6B42F01E
:1029C00080025A635A6D42F080025A655A6D5A6904
:1029D00042F080025A615A6922F080025A610E2147
:1029E00043205B69FEF73CFC1E4BE3601E4BC4F8C2
:1029F00000380023C4F8003EC0232360EE6E4FF47D
:102A00000413A3633369002BFCDA012333610C2028
:102A100000F03EFE3369DB07FCD4122000F038FEE4
:102A20003369002BFCDA0026A6602846FFF740FF3A
:102A30006B68C4F81068DB68C4F81468C4F81C68D4
:102A40004BB90A4BA3614FF0FF336361A36843F0B6
:102A50000103A36070BD064BF4E700BF50320220B3
:102A6000003802404014004003002002003C30C007
:102A7000083C30C0F8B5C46E054600212046FFF77B
:102A800035FF296F00234FF001128F68C4F83438E6
:102A90004FF00066C4F81C284FF0FF3004EB4312DF
:102AA00001339F42C2F80069C2F8006BC2F80809FE
:102AB000C2F8080BF2D20B68EA6E6B6763621023F0
:102AC0001361166916F01006FBD1122000F0E0FD2C
:102AD000D4F8003823F4FE63C4F80038A36943F443
:102AE000402343F01003A3610923C4F81038C4F84D
:102AF00014380A4BEB604FF0C043C4F8103B084B4E
:102B0000C4F8003BC4F81069C4F800396B6F03F1D6
:102B1000100243F480136A67A362F8BDB83D000851
:102B200040800010C26E90F86610D2F8003823F48E
:102B3000FE6343EA0113C2F8003870472DE9F04103
:102B40000EB200EB86080D46D8F80C100F6807F09F
:102B50000303022B50D0032B50D03D4A3D4F012B95
:102B600018BF1746C46E4FEA451E04EB0E03002241
:102B7000C3F8102B8A6905F1100C002A40D04A8A4C
:102B800005F158035B013A43E2500123D4F81C28B5
:102B900003FA0CF31343A6444A69C4F81C38002313
:102BA000CEF8103905F13F03002A39D00A8A898B03
:102BB0009208012988BF4A43416F04EB83035618EA
:102BC00041EA0242466729465A602046FFF78EFED8
:102BD000D8F80C301B8A43EA85531F4305F148039C
:102BE0005B01E7500123D4F81C2803FA05F51543CF
:102BF000C4F81C58BDE8F081174FB3E7174FB1E791
:102C000004EB4613D3F8002B22F40042C3F8002B48
:102C1000D4F81C28012303FA0CF322EA0303BAE7D1
:102C200004EB83030E4A5A6004EB461629462046FD
:102C3000FFF75CFED6F8003923F40043C6F80039EC
:102C4000D4F81C38012202FA05F523EA0505CFE77E
:102C500000800010008004100080081000800C101C
:102C600000040002026F12684267FFF721BE0000F5
:102C70005831C36E49015B5813F4004004D013F47B
:102C8000001F14BF01200220704700004831C36EAE
:102C900049015B5813F4004004D013F4001F14BF23
:102CA000012002207047000000EB8101CB68196A07
:102CB0000B6813604B6853607047000000EB8103A2
:102CC00030B5DD68AA691368D36019B9402B84BF99
:102CD000402313606B8A1468C26E1C44013CB4FB31
:102CE000F3F46343033323F0030302EB411043EA9D
:102CF000C44343F0C043C0F8103B2B6803F0030308
:102D0000012B09B20ED1D2F8083802EB411013F4AE
:102D1000807FD0F8003B14BF43F0805343F0005352
:102D2000C0F8003B02EB4112D2F8003B43F00443F1
:102D3000C2F8003B30BD00002DE9F041244DEE6E9D
:102D400006EB40130446D3F8087BC3F8087B38072A
:102D50000AD5D6F81438190706D505EB84032146A1
:102D6000DB6828465B689847FA072FD5D6F81438F1
:102D7000DB072BD505EB8403D968CCB98B69488A6E
:102D80005E68B6FBF0F200FB12628AB91868DA6876
:102D900090420DD2121A83E81400202383F3118885
:102DA0000B482146FFF78AFF84F31188BDE8F081C4
:102DB000012303FA04F26B8923EA02036B81CB68D7
:102DC00023B121460248BDE8F0411847BDE8F08133
:102DD0005032022000EB810370B5DD68C36E6C6970
:102DE0002668E6604A0156BB1A444FF40020C2F838
:102DF00010092A6802F00302012A0AB20ED1D3F8A0
:102E0000080803EB421410F4807FD4F8000914BFC3
:102E100040F0805040F00050C4F8000903EB42122B
:102E2000D2F8000940F00440C2F80009D3F8340891
:102E3000012202FA01F10143C3F8341870BD19B937
:102E4000402E84BF4020206020682E8A841940F0E4
:102E50000050013C1A44B4FBF6F440EAC440C6E713
:102E6000F8B504461E48C56E05EB4413D3F808694F
:102E7000C3F80869F10717D5D5F81038DA0713D564
:102E800000EB8403D9684B691F68DA68974218D24F
:102E9000D21B00271A605F60202383F3118821462C
:102EA000FFF798FF87F31188330617D5D5F8342834
:102EB0000123A340134211D02046BDE8F840FFF79C
:102EC0001FBD012303FA04F2038923EA02030381ED
:102ED0008B68002BE8D021469847E5E7F8BD00BF96
:102EE00050320220A0482DE9F84FC56E6E69AB69DB
:102EF0001E4016F4805F6E61044605D0FEF7A2FD09
:102F0000BDE8F84FFFF748BC002E12DAD5F8003EB6
:102F100095489B071EBFD5F8003E23F00303C5F874
:102F2000003ED5F8043823F00103C5F80438FEF755
:102F3000B5FD370502D58C48FEF7A4FDB0040CD5CD
:102F4000D5F8083813F0060FEB6823F470530CBF64
:102F500043F4105343F4A053EB60310704D5636886
:102F6000DB680BB180489847F2026FD4B3020CD5EE
:102F7000D4F86C80DFF8F0A100274FF00109236F2F
:102F80009B68F9B28B4280F09C80F70619D5E16E00
:102F90000A6AC2F30A1702F00F0302F4F012B2F544
:102FA000802F00F0B680B2F5402F0AD104EB8303E6
:102FB00001F58051DB68186A00231A469F4240F0F1
:102FC0009C803303D5F818481DD5E70302D50020AF
:102FD000FFF7B2FEA50302D50120FFF7ADFE6003A7
:102FE00002D50220FFF7A8FE210302D50320FFF738
:102FF000A3FEE20202D50420FFF79EFEA30202D543
:103000000520FFF799FE77037FF57AAFE60702D533
:103010000020FFF725FFA50702D50120FFF720FFBD
:10302000600702D50220FFF71BFF210702D503200E
:10303000FFF716FFE20602D50420FFF711FFA306F3
:103040007FF55EAF0520FFF70BFF59E7D4F86C80E2
:10305000DFF814A100274FF00109236F9B685FFA86
:1030600087FB5B4582D308EB4B13D3F8002902F4AE
:103070004022B2F5802F22D1D3F80029002A1EDA8F
:10308000D3F8002942F09042C3F80029D3F8002970
:10309000002AFBDB5946E06EFFF728FC228909FA7B
:1030A0000BF322EA0303238104EB8B03DB689B68A9
:1030B00013B15946504698475846FFF721FC01374F
:1030C000CBE708EB4112D2F8003B03F44023B3F501
:1030D000802F10D1D2F8003B002B0CDA628909FA5C
:1030E00001F322EA0303638104EB8103DB68DB68FD
:1030F0000BB150469847013741E79C0708BF0A6863
:10310000072B98BF027003F101039CBF120A013024
:1031100054E7023304EB830201F580515268906951
:103120000268D0F808C04068A2EB000E00221046EA
:1031300097420AD104EB830463689B699A683A4416
:103140009A605A6817445F603BE712F0030F08BFAC
:103150000868964588BF8CF8000002F1010284BF20
:10316000000A0CF1010CE3E750320220C36E03EBBE
:103170004111D1F8003B43F40013C1F8003B704704
:10318000C36E03EB4111D1F8003943F40013C1F8C9
:1031900000397047C36E03EB4111D1F8003B23F4B3
:1031A0000013C1F8003B7047C36E03EB4111D1F827
:1031B000003923F40013C1F80039704730B5039C7F
:1031C0000172043304FB0325C361049B03630021E4
:1031D000059B00604060C1604261026185610462DC
:1031E00042628162C162436330BD00000022416AD5
:1031F00041610161C2608262C2626FF00101FEF74B
:103200006DBF000003694269934203D1C2680AB1ED
:1032100000207047181D704703691960C2680132A9
:10322000C260C269134482690361934224BF436A46
:1032300003610021FEF746BF38B504460D46E3683A
:103240003BB16269131D1268A3621344E36200205C
:1032500038BD237A33B929462046FEF723FF0028DC
:10326000EDDA38BD6FF00100FBE70000C368C2690A
:10327000013BC3604369134482694361934224BFA5
:10328000436A436100238362036B03B118477047AD
:1032900070B52023044683F31188866A3EB9FFF790
:1032A000CBFF054618B186F31188284670BDA36A86
:1032B000E26A13F8015BA362934202D32046FFF750
:1032C000D5FF002383F31188EFE700002DE9F84FC5
:1032D00004460E4690469946202787F3118800251C
:1032E000AA46D4F828B0BBF1000F09D149462046C0
:1032F000FFF7A2FF20B18BF311882846BDE8F88FB5
:10330000A16AE36AA8EB050B5B1A9B4528BF9B46A5
:10331000BBF1400F1BD9334601F1400251F8040BB9
:1033200043F8040B9142F9D1A36A40334036A362BB
:103330004035A26AE36A9A4202D32046FFF796FF1D
:103340008AF311884545D8D287F31188C9E73046FA
:103350005A46FDF77BFDA36A5B445E44A3625D446D
:10336000E7E7000010B5029C0172043303FB04215F
:10337000C36100238362C362039B0363049B0060F9
:103380004060C460426102618161046242624363E1
:1033900010BD0000026AC260426A426102610022FE
:1033A0008262C2626FF00101FEF798BE4369026952
:1033B0009A4203D1C2680AB100207047184650F8FB
:1033C000043B0B6070470000C368C2690133C360EF
:1033D0004369134482694361934224BF436A436152
:1033E0000021FEF76FBE000038B504460D46E368C5
:1033F0003BB123691A1DA262E2691344E362002013
:1034000038BD237A33B929462046FEF74BFE002803
:10341000EDDA38BD6FF00100FBE7000003691960C9
:10342000C268013AC260C26913448269036193426F
:1034300024BF436A036100238362036B03B118470F
:103440007047000070B5202304460E4683F31188B0
:10345000856A35B91146FFF7C7FF10B185F31188AA
:1034600070BDA36A1E70A36AE26A01339342A3622D
:1034700004D3E16920460439FFF7D0FF002080F330
:10348000118870BD2DE9F84F04460D4691469A46C5
:103490004FF0200888F311880026B346A76A4FB979
:1034A00051462046FFF7A0FF20B187F31188304630
:1034B000BDE8F88FA06AE76AA9EB06033F1A9F42AE
:1034C00028BF1F46402F1BD905F1400355F8042B98
:1034D00040F8042B9D42F9D1A36A4033A3624036E1
:1034E000A26AE36A9A4204D3E16920460439FFF7ED
:1034F00095FF8BF311884E45D9D288F31188CDE71B
:1035000029463A46FDF7A2FCA36A3B443D44A36228
:103510003E44E5E7026943699A4203D1C3681BB997
:10352000184670470023FBE7836A002BF8D0043B62
:103530009B1AF5D01360C368013BC360C3691A448A
:10354000836902619A4224BF436A03610023836254
:103550000123E5E700F042B94FF0804300225863B1
:103560001A610222DA6070474FF080430022DA606D
:10357000704700004FF0804358637047FEE700003B
:1035800010B5194CFEF794FCFEF7B6FD80221749E2
:103590002046FEF73BFD012344F8180C0374144B3E
:1035A000144AD96821F4E0610904090C0A4312495C
:1035B000DA60CA6842F08072CA60104A1049C2F8E4
:1035C000B01F116841F0010111601022DA7720224A
:1035D00083F82220002383F3118862B60948BDE8EE
:1035E0001040FEF735BD00BFDC2A0220E83D000890
:1035F00000ED00E00003FA05F0ED00E0001000E04F
:1036000055CEACC5F03D00082DE9F84F1F4C4FF0EA
:103610000008656904F11407C1464FF08043266A2B
:103620005B6AAA689E1B96421DD34FF0200AAA68C7
:10363000236AD5F80CB0134423622B68BB425F6049
:10364000A6EB02066361C5F80C8001D1FFF78CFF81
:1036500089F311882869D8478AF311886569AB68AE
:103660009E42E4D2D9E76269BA420CD091682362E3
:103670008E1B9660A86802282CBF1818981CBDE8FD
:10368000F84FFFF777BFBDE8F88F00BFB42A0220DC
:10369000034B59685A68521A9042FBD8704700BFD2
:1036A000001000E04B6843608B688360CB68C360A8
:1036B0000B6943614B6903628B6943620B6803606A
:1036C0007047000008B5274B27481A6940F2FF7180
:1036D0000A431A611A6922F4FF6222F007021A6192
:1036E0001A691A6B0A431A631A6D0A431A651F4A4C
:1036F0001B6D1146FFF7D6FF1D4802F11C01FFF7B5
:10370000D1FF1C4802F13801FFF7CCFF1A4802F143
:103710005401FFF7C7FF194802F17001FFF7C2FF1C
:10372000174802F18C01FFF7BDFF164802F1A8010E
:10373000FFF7B8FF144802F1C401FFF7B3FF1348C5
:1037400002F1E001FFF7AEFF114802F1FC01FFF7C3
:10375000A9FF104802F58C71FFF7A4FFBDE80840EF
:1037600000F09EB80038024000000240103E000801
:103770000004024000080240000C02400010024019
:103780000014024000180240001C024000200240C9
:10379000002402400028024008B500F0F5F9FFF7C8
:1037A000EFFEFEF7D7FFBDE80840FEF7AFBD000013
:1037B000704700004FF0804310B51A69920708D592
:1037C00000241C61202383F31188FFF71DFF84F37D
:1037D0001188BDE81040FEF7DFBF0000104B1A6CE7
:1037E00042F001021A641A6E42F001021A660D4A92
:1037F0001B6E936843F0010393604FF080436B228C
:103800009A624FF0FF32DA6200229A615A63DA60FC
:103810005A6001225A6108211A601C20FDF720BD60
:1038200000380240002004E01B4B1A696FEA425244
:103830006FEA52521A611A69C2F30A021A614FF012
:10384000FF301A695A69586100215A6959615A69E9
:103850001A6A62F080521A621A6A02F080521A6280
:103860001A6A5A6A58625A6A59625A6A0B4A106846
:1038700040F480701060186F00F44070B0F5007F65
:103880001EBF4FF4803018671967536823F4007324
:10389000536000F059B900BF00380240007000408A
:1038A000354B364A1A64364A4FF4404111601A6863
:1038B00042F001021A601A689207FCD59A6822F059
:1038C00003029A602C4B19469A6812F00C02FBD145
:1038D000186800F0F90018609A601A6842F48032A3
:1038E0001A600B689B03FCD54B6F43F001034B67D9
:1038F000214B5A6F9007FCD5224A5A601A6842F051
:1039000080721A601E4B1A4659684904FCD5196822
:1039100041F4803119605368D803FCD5136843F42F
:1039200000331360164A53689903FCD5124B1A688A
:103930009201FCD5144A9A6040F20112C3F88C201F
:103940000022C3F89020114A40F2073111609A68B2
:1039500042F002029A60084B9A6802F00C02082AB0
:10396000FAD15A6C42F480425A645A6E42F4804250
:103970005A665B6E704700BF0038024000040010BA
:1039800000700040086C400900948838003C0240F8
:10399000084A08B5536911680B4003F001035361ED
:1039A00023B1054A13680BB150689847BDE8084039
:1039B000FEF7F2BE003C0140C8250220084A08B5C7
:1039C000536911680B4003F00203536123B1054AA8
:1039D00093680BB1D0689847BDE80840FEF7DCBE9D
:1039E000003C0140C8250220084A08B55369116807
:1039F0000B4003F00403536123B1054A13690BB173
:103A000050699847BDE80840FEF7C6BE003C01403B
:103A1000C8250220084A08B5536911680B4003F015
:103A20000803536123B1054A93690BB1D0699847E4
:103A3000BDE80840FEF7B0BE003C0140C8250220AA
:103A4000084A08B5536911680B4003F0100353612D
:103A500023B1054A136A0BB1506A9847BDE8084084
:103A6000FEF79ABE003C0140C8250220174B10B556
:103A70005C691A68144004F478725A61A30604D58C
:103A8000134A936A0BB1D06A9847600604D5104A6E
:103A9000136B0BB1506B9847210604D50C4A936BFE
:103AA0000BB1D06B9847E20504D5094A136C0BB1F2
:103AB000506C9847A30504D5054A936C0BB1D06CA4
:103AC0009847BDE81040FEF767BE00BF003C0140CC
:103AD000C82502201A4B10B55C691A68144004F41A
:103AE0007C425A61620504D5164A136D0BB1506DC4
:103AF0009847230504D5134A936D0BB1D06D9847B1
:103B0000E00404D50F4A136E0BB1506E9847A10420
:103B100004D50C4A936E0BB1D06E9847620404D55D
:103B2000084A136F0BB1506F9847230404D5054A18
:103B3000936F0BB1D06F9847BDE81040FEF72CBED5
:103B4000003C0140C8250220062108B50846FDF7C3
:103B500087FB06210720FDF783FB06210820FDF7E0
:103B60007FFB06210920FDF77BFB06210A20FDF7DC
:103B700077FB06211720FDF773FB06212820BDE8FF
:103B80000840FDF76DBB000008B5FFF74DFEFDF7DF
:103B900045FAFDF70BFDFDF7E1FEFDF7B5FDFFF77B
:103BA00007FEBDE80840FFF7D5BC0000034611F84A
:103BB000012B03F8012B002AF9D1704712101213C0
:103BC000121100000010410001105A00F42A0220D6
:103BD0004826022053544D3332463F3F3F3F3F3F3C
:103BE0000053544D333246375B347C355D78005397
:103BF000544D333246375B367C375D780000000029
:103C0000009600000000000000000000000000001E
:103C10000000000000000000000000007515000812
:103C2000611500089D150008891500089515000804
:103C3000811500086D15000859150008A915000820
:103C400000000000811600086D160008A916000883
:103C500095160008A11600088D16000879160008B0
:103C600065160008051700080000000001000000AC
:103C7000000000000200000000000000AD18000875
:103C800015190008400040008C2F02209C2F0220B4
:103C9000020000000000000003000000000000001F
:103CA000591900080000000010000000AC2F02208D
:103CB000000000000100000000000000503202205F
:103CC000010102004172647550696C6F74002542F5
:103CD0004F415244252D424C002553455249414CF9
:103CE00025000000AD220008152200081918000860
:103CF0009122000843000000FC3C00080902430038
:103D0000020100C032090400000102020100052482
:103D1000001001052401000104240202052406000C
:103D200001070582030800FF09040100020A0000E0
:103D30000007050102400000070581024000000065
:103D400012000000483D000812011001020000406E
:103D50000912415700020102030100000403090493
:103D600025424F41524425004D6174656B463736FC
:103D7000352D57696E670030313233343536373878
:103D80003941424344454600008000000080000065
:103D9000008000000080000000000200000004001D
:103DA0000000040000000400000004000000040003
:103DB000000004000000040000000000B11A000828
:103DC000911D00083D1E000840004000C83202203E
:103DD000C832022001000000D8320220800000001A
:103DE00040010000050000006D61696E00000000E8
:103DF000083E0008E0320220D83402200100000012
:103E00007D3500080000000069646C65000000005A
:103E10000000802A00000000AAAAAAAA0000000050
:103E2000FFFF00000000000000A00A0000000000EA
:103E300000000000AAAAAAAA00000000FFFF0000DC
:103E40000000000000000000000000000000000072
:103E5000AAAAAAAA00000000FFFF000000000000BC
:103E6000000000000000100000000000AAAAAAAA9A
:103E700000000000FFFB0000000000000000000048
:103E80000080020000000000AAAAAAAA00400100C7
:103E9000FFFF00000000008008000000000000009C
:103EA00000000000AAAAAAAA00000000FFFF00006C
:103EB0000000000000000000000000000000000002
:103EC000AAAAAAAA00000000FFFF0000000000004C
:103ED000000000000000000000000000AAAAAAAA3A
:103EE00000000000FFFF00000000000000000000D4
:103EF0000000000000000000AAAAAAAA000000001A
:103F0000FFFF0000000000000000000000000000B3
:103F100000000000000000000000000000000000A1
:103F20000000000000000000000000000000000091
:103F30000000000000000000000000000000000081
:103F40000000000000000000FF0000000000000072
:103F5000D43B00083F00000049040000E13B00089A
:103F60003F00000051040000EF3B00083F0000004C
:103F70000096000000000800040000005C3D0008FE
:103F80000000000000000000000000000000000031
:083F9000000000000000000029
:00000001FF
